:020000020000FC
:080000000C94CD090C94F708E3
:040014000C945509EA
:04001C000C94BD097A
:04002C000C947909AE
:040038000C941B0900
:040048000C945B17A2
:100050000C942B17003B19EB0C3BA9EBD00005C30C
:10006000000035C3E00082C30000BEC3420105AA00
:10007000000035AAAE0182AA0000B2AAC000059114
:10008000C6008291B201057800005978CC008278D0
:100090000000B278D400055F0000355FD800825FB1
:1000A0000000D65F1001054600004146BA018246B5
:1000B0000000CA462801052D0000412DC701051486
:1000C000426F6F74000044656D6F000043616C0007
:1000D0004E756D004C6564004275726E696E00006D
:1000E0004469616C00004F6E00004F66660031325B
:1000F000687200003234687200004865780044611C
:100100007465000042696E00526F6D004D696E00AB
:10011000506C617900004E6F726D00005265760080
:1001200046460000465200004E616D650000456481
:10013000697400005075736820546F2053746172A5
:100140007400475053004F6666002D3132002D3148
:1001500031002D3130002D3920002D3820002D3771
:1001600020002D3620002D3520002D3420002D3389
:1001700020002D3220002D312000302020002B3196
:1001800020002B3220002B3320002B3420002B3575
:1001900020002B3620002B3720002B3820002B3955
:1001A00020002B3130002B3131002B3132004453F1
:1001B00054004368726F6E6F00005265736574007F
:1001C0004A64520077007A0084008200860077003B
:1001D0007A007D007F007500750073008B008E0033
:1001E00090009200730075009700F800FA00750007
:1001F000555341004555000044656D6F2000420095
:1002000050004700F81206135401E212F0125C018C
:10021000EB13FF1364012914391468010117381214
:100220006C012C1C3812740142144F147C011513FC
:100230001F138401261330138C01381342139401C9
:100240004A1358139C0158146514A4015F137013CA
:10025000A8017E13A7130000292AC11101802A2BAF
:10026000D51102802B2CCE1103802CB1C7110000B8
:100270002D2EC21118012E2FD51110012F30CE11A5
:10028000080130B1C71100003C3DC21118413D3E8C
:10029000D51110413E3FCE1108413FB1C7110000BA
:1002A0004243C11105804341F611048041C5F41158
:1002B00000004540EC11018040C4EA1100004428D0
:1002C000F81100003132C311200132B3DD110000FA
:1002D0003300E11100009281E7D6B4A392005140AF
:1002E0003625036251000CF80C46F846F8F80CF875
:1002F000FF0001FE0101FE01FEFE01FEFE01010103
:10030000FEFE01FE0101FE01FEFEFF0089018D01DE
:1003100091010B694F0B8C4FFF000B697F0B8C4FCA
:10032000FF000B694F0B8C7FFF009B01A001A50113
:10033000AA01AF01B4010B694F0B8C4F0BAF4FFFFC
:100340000B697F0B8C4F0BAF4FFF0B694F0B8C7FF3
:100350000BAF4FFF0B697F0B8C7F0BAF4FFF0B6910
:100360004F0B8C4F0BAF7FFF0B697F0B8C4F0BAF8D
:100370007FFFC301CA01D101D801DF01E601ED0110
:10038000F401FB0102020B694F0B8C4F0BAF4F0BBB
:10039000D24FFF000B697F0B8C4F0BAF4F0BD24F2F
:1003A000FF000B694F0B8C7F0BAF4F0BD24FFF0041
:1003B0000B697F0B8C7F0BAF4F0BD24FFF000B698C
:1003C0004F0B8C4F0BAF7F0BD24FFF000B697F0B96
:1003D0008C4F0BAF7F0BD24FFF000B694F0B8C7F05
:1003E0000BAF7F0BD24FFF000B697F0B8C7F0BAFE6
:1003F0007F0BD24FFF000B694F0B8C4F0BAF4F0B96
:10040000D27FFF000B697F0B8C4F0BAF4F0BD27F5E
:10041000FF003031323334353637383941424344C6
:1004200045460C0102030405060708090A0B0C01E6
:1004300002030405060708090A0B00000100010178
:100440000001FF01FF00FFFF00FF4A616E1F4665CC
:10045000621C4D61721F4170721E4D61791F4A7599
:100460006E1E4A756C1F4175671F5365701E4F6382
:10047000741F4E6F761E4465631F80FE80F2008DF0
:10048000FE8CF9009AFC99F700A6F8A5F400B3F4E5
:10049000B1EF00BFEEBAE500CAE6C7E200D4DED095
:1004A000DA00DDD5D9D100E5CBE1C800EDBFE4BA73
:1004B00000F3B4EEB200F7A7F3A600FB9BF69A0098
:1004C000FD8EF88D00FD80F18000FD73F87400FB57
:1004D00066F66700F75AF35B00F34DEE4F00ED410F
:1004E000E44600E536E13900DD2CD93000D423D0D4
:1004F0002700CA1BC71F00BF13BA1C00B30DB112DF
:1005000000A609A50D009A05990A008D038C080024
:100510007F037F0F0072037308006505660A0059A8
:10052000095A0D004C0D4E12004113461C00351B9C
:10053000381F002B232F2700222C2630001A361EAE
:10054000390012421B47000C4D114F00085A0C5B3A
:10055000000466096700027307740002810E8100BF
:10056000028E078D00049B099A0008A70CA6000CB8
:10057000B411B20012BF1BBA001ACB1EC80022D59C
:1005800026D1002BDE2FDA0035E638E20040EE45BA
:10059000E5004CF44EEF0059F85AF40065FC66F79C
:1005A0000072FE73F9FF7AEB7AD90080E883EB8959
:1005B000EB8CE88CE580D98CD900B5E4B5D200008D
:1005C000D2BBD5BEDBBEDEBBDEB8D2ACDEAC00003B
:1005D000E286E589EB89EE86EE83EB80EE7DEE7AAE
:1005E000EB77E577E27A00E580EB8000E04CD44CD5
:1005F000DD55DD430000B831AC31AC28B528B82555
:10060000B822B51FAF1FAC220000852182247C24B4
:10061000792179157C12821285158518821B7C1B25
:1006200079180047315331532E502B4D254D1F0063
:10063000224C1F4F1F52225528552B522B4F284C0E
:10064000224C1F491F46224328432B462B49284C46
:1006500000001D841A811A81148111841187148A63
:100660001A8A1D871D7B1A781478117B000021BE21
:1006700021AC000027BB2ABE30BE33BB33AF30AC49
:100680002AAC27AF27BB000049E449D2000053E45D
:1006900053D2FF0073EF76F27CF27FEF7FEC73E0D2
:1006A0007FE0008DE981E98AF28AE000AAE2AAD01F
:1006B0000000B0DFB3E2B9E2BCDFBCDCB9D9BCD624
:1006C000BCD3B9D0B3D0B0D300B3D9B9D900D0BC62
:1006D000D0AA0000E2B3D6B3DFBCDFAA0000DC89F9
:1006E000DC7700EE89E289E280EB80EE7DEE7AEB4A
:1006F00077E577E27A00D055D0430000E252DF552B
:10070000D955D652D646D943DF43E246E249DF4CBB
:10071000D94CD6490000AA2DAA1B0000B02DBC2D33
:10072000BC2AB927B621B61B00007B217B0F0083B2
:1007300018801B801E832189218C1E8C1B891883A5
:100740001880158012830F890F8C128C1589180060
:10075000492F491D00005B295826582652264F294B
:100760004F2C522F582F5B2C5B20581D521D4F20B1
:1007700000001E52215527552A522A4F1E432A4354
:1007800000002F52325538553B523B4638433243D6
:100790002F462F5200001187148A1A8A1D871D8444
:1007A00011781D780000238A237800001EBB21BE2B
:1007B00027BE2ABB2AB81EAC2AAC00002FBB32BE13
:1007C00038BE3BBB3BB82FAC3BAC000040DD43E048
:1007D00049E04CDD4CDA40CE4CCE000051DD54E017
:1007E0005AE05DDD5DDA5AD75DD45DD15ACE54CE84
:1007F00051D10054D75AD7FF76DF8ADF0079DF80E6
:10080000F30079F380DF0083DF83F30087F387DF72
:100810000076F38AF300ADD1B5D100B1D1B1E500D6
:10082000ADE5B5E50000D2ABDEAB00D6ABD6BF0080
:10083000DAABDABF00D2BFDEBF00DC76EE7600E0D6
:1008400076E08A00E576E58A00EA76EA8A00DC8AC4
:10085000EE8A00CA42DE4200CE42CE5600D356D7C0
:1008600042DB5600CA56DE560000A922B92200AD6E
:1008700036B122B53600A936B93600007514891490
:100880000079287D14812800851485280075288921
:100890002800432259220046364A224E3600512271
:1008A00051360055225536004336593600001D4258
:1008B000394200225626422A56002E422E56003237
:1008C0004232560036423656001D563956001177D0
:1008D0002377001477148B001877208B00188B2057
:1008E0007700118B238B000024AB32AB0027AB2F9A
:1008F000BF0027BF2FAB0024BF32BF0048D15AD161
:10090000004BD153E5004BE553D10056D156E500DD
:1009100048E55AE5FF007AEB7AD90080E883EB8955
:10092000EB8CE88CE580D98CD900E286E589EB89EF
:10093000EE86EE83EB80EE7DEE7AEB77E577E27A7A
:1009400000E580EB8000852182247C2479217915C3
:100950007C12821285158518821B7C1B7918001D5C
:10096000841A811A81148111841187148A1A8A1DAC
:10097000871D7B1A781478117BFF80EC8080FF8BB9
:10098000EC8080FF96EA8080FFA1E78080FFABE3E8
:100990008080FFB6DE8080FFBFD88080FFC8D18016
:1009A00080FFD0C98080FFD7C08080FFDDB6808007
:1009B000FFE2AC8080FFE6A28080FFE9978080FFA5
:1009C000EB8C8080FFEB808080FFEB758080FFE9FF
:1009D0006A8080FFE65F8080FFE2558080FFDD4A0D
:1009E0008080FFD7418080FFD0388080FFC8308072
:1009F00080FFBF298080FFB6238080FFAB1E8080F0
:100A0000FFA11A8080FF96178080FF8B158080FFE2
:100A100080158080FF74158080FF69178080FF5EDD
:100A20001A8080FF541E8080FF4A238080FF402967
:100A30008080FF37308080FF2F388080FF28418002
:100A400080FF224B8080FF1D558080FF195F8080D2
:100A5000FF166A8080FF14758080FF14808080FFFD
:100A6000148C8080FF16978080FF19A28080FF1D64
:100A7000AC8080FF22B68080FF28C08080FF2FC915
:100A80008080FF37D18080FF40D88080FF49DE80A2
:100A900080FF54E38080FF5EE78080FF69EA80800A
:100AA000FF74EC8080FF828080E67E808280FF8100
:100AB000808AE67E818180FF818095E47E818180CD
:100AC000FF81809FE27E818180FF8180A9DE7E811F
:100AD0008180FF817FB3D97E82817FFF817FBBD3FD
:100AE0007E82817FFF817FC4CC7E82817FFF817F78
:100AF000CBC57E82817FFF817FD2BC7E82817FFFDA
:100B0000807FD8B37F82807FFF807FDDAA7F828055
:100B10007FFF807FE1A07F82807FFF807FE3967FE1
:100B200082807FFF807FE58B7F82807FFF7F7EE5F5
:100B30008080827F7EFF7F7FE57680827F7FFF7F60
:100B40007FE36B80827F7FFF7F7FE16180827F7F99
:100B5000FF7F7FDD5780827F7FFF7E7FD84D818240
:100B60007E7FFF7E7FD24581827E7FFF7E7FCB3C72
:100B700081827E7FFF7E7FC43581827E7FFF7E7F84
:100B8000BB2E81827E7FFF7E7FB32881827E7FFFA6
:100B90007E80A92381817E80FF7E809F1F81817E50
:100BA00080FF7E80951D81817E80FF7E808A1B81F3
:100BB000817E80FF7E817F1B82807E81FF7E8175AA
:100BC0001B81807E81FF7E816A1D81807E81FF7E08
:100BD00081601F81807E81FF7E81562381807E819E
:100BE000FF7E814D2881807E81FF7E82442E817F21
:100BF0007E82FF7E823B35817F7E82FF7E82343C17
:100C0000817F7E82FF7E822D45817F7E82FF7F8273
:100C1000274E807F7F82FF7F822257807F7F82FFE7
:100C20007F821E61807F7F82FF7F821C6B807F7F3F
:100C300082FF7F821A76807F7F82FF80821A817F87
:100C40007E8082FF80821A8B7F7F8082FF80821C61
:100C5000967F7F8082FF80821EA07F7F8082FF80C0
:100C60008222AA7F7F8082FF808227B37F7F80825B
:100C7000FF81822DBC7E7F8182FF818234C57E7F91
:100C80008182FF81823BCC7E7F8182FF818244D33F
:100C90007E7F8182FF81824CD97E7F8182FF81812C
:100CA00056DE7E808181FF818160E27E808181FFCE
:100CB00081816AE47E808181FF818175E67E808109
:100CC00081FF828080BC7E808280FF818086BC7EA6
:100CD000818180FF81808CBB7E818180FF818092B9
:100CE000BA7E818180FF818098B77E818180FF817B
:100CF0007F9EB47E82817FFF817FA3B17E82817FD0
:100D0000FF817FA8AD7E82817FFF817FACA97E823B
:100D1000817FFF817FB0A47E82817FFF807FB39E31
:100D20007F82807FFF807FB6997F82807FFF807F78
:100D3000B9937F82807FFF807FBA8D7F82807FFF23
:100D4000807FBB877F82807FFF7F7EBB8080827FAA
:100D50007EFF7F7FBB7A80827F7FFF7F7FBA748038
:100D6000827F7FFF7F7FB96E80827F7FFF7F7FB62C
:100D70006880827F7FFF7E7FB36281827E7FFF7E7D
:100D80007FB05D81827E7FFF7E7FAC5881827E7FD7
:100D9000FF7E7FA85481827E7FFF7E7FA350818269
:100DA0007E7FFF7E7F9E4D81827E7FFF7E80984A80
:100DB00081817E80FF7E80924781817E80FF7E8060
:100DC0008C4681817E80FF7E80864581817E80FF8A
:100DD0007E817F4582807E81FF7E81794581807E14
:100DE00081FF7E81734681807E81FF7E816D478198
:100DF000807E81FF7E81674A81807E81FF7E816265
:100E00004D81807E81FF7E825C50817F7E82FF7E6D
:100E1000825754817F7E82FF7E825358817F7E82FB
:100E2000FF7E824F5D817F7E82FF7F824C63807F69
:100E30007F82FF7F824968807F7F82FF7F82466E4C
:100E4000807F7F82FF7F824574807F7F82FF7F82E9
:100E5000447A807F7F82FF808244817F7E8082FF10
:100E6000808244877F7F8082FF8082458D7F7F8064
:100E700082FF808246937F7F8082FF808249997FB4
:100E80007F8082FF80824C9E7F7F8082FF81824FA5
:100E9000A47E7F8182FF818253A97E7F8182FF8130
:100EA0008257AD7E7F8182FF81825CB17E7F8182AD
:100EB000FF818261B47E7F8182FF818167B77E80FE
:100EC0008181FF81816DBA7E808181FF818173BBC9
:100ED0007E808181FF818179BC7E808181FF103895
:100EE0003810100010006C6C480000000000002852
:100EF0007C28287C2800203840300870100064646A
:100F00000810204C4C002050502054483400303001
:100F100020000000000010202020202010002010C1
:100F20001010101020000028387C38280000001015
:100F3000107C101000000000000000303020000085
:100F400000780000000000000000003030000004C5
:100F500008102040000038444C54644438001030DD
:100F60001010101038003844041820407C00384419
:100F7000043804443800081828487C0808007C40DD
:100F800040780444380018204078444438007C04F9
:100F900008102020200038444438444438003844A5
:100FA000443C040830000000606000606000000005
:100FB00030300030302008102040201008000000A1
:100FC0007C00007C00002010080408102000384439
:100FD00004181000100038445C545C403800384459
:100FE00044447C4444007844447844447800384481
:100FF00040404044380078444444444478007C40B5
:10100000407840407C007C4040784040400038447C
:10101000405C44443C004444447C44444400381014
:1010200010101010380004040404444438004448EC
:101030005060504844004040404040407C00446C78
:101040005444444444004464544C444444003844AC
:101050004444444438007844447840404000384494
:101060004444544834007844447848444400384464
:101070004038044438007C10101010101000444414
:101080004444444438004444444444281000444404
:1010900054545454280044442810284444004444E0
:1010A00044281010100078081020404078003820A4
:1010B00020202020380000402010080400003808BC
:1010C000080808083800102844000000000000004C
:1010D0000000000000FC30301000000000000000A4
:1010E00038043C443C0040407844444478000000CC
:1010F00038444044380004043C4444443C0000006C
:101100003844784038001820207820202000000043
:101110003C44443C04384040704848484800100073
:101120001010101018000800180808084830404037
:1011300048506050480010101010101018000000A7
:101140006854544444000000704848484800000077
:101150003844444438000000784444447840000057
:101160003C4444443C04000058242020700000000B
:101170003840380438000020782020281000000073
:101180004848485828000000444444281000000003
:101190004444547C2800000048483048480000007F
:1011A000484848381060000078083040780018201F
:1011B00020602020180010101000101010003008BF
:1011C000080C080830002850000000000000387C9F
:1011D0007C7C7C7C38005A9A0E941D1802E0109199
:1011E000F30210FD03E000936900E89A08950F935D
:1011F0000FB70F9300918704002311F09460F882D9
:101200000F910FBF0F9118950F93F4BC05E005BD2A
:101210000FE707BD0F9108950DE70B8F08959260BA
:10122000FB8E02E005BB02E000936E00089500E033
:1012300000936E0008950F93F6BC78940FB70F9348
:101240001F930B8D002349F00A950B8F31F4009109
:10125000FD02002311F49860FE8E0F8D000F1E2DED
:101260001C9B1127012B0F8F003849F40E8D0E1592
:10127000A1F00FAD08600FAFEE8ECEDF0EC00F37BE
:1012800021F00F3F51F40ED008C00E8D002329F03D
:101290009062FE8E0FAD077F0FAF1F910F910FBFB2
:1012A0000F9118959D7FC3DF0895FFCF04E0009351
:1012B000810005E00093890006E10093880013D0C7
:1012C000089508E017E0F8940C8F1D8F7894089526
:1012D00000EF10E0F8CF1F930C8D1D8D012B09F04E
:1012E0000E2D1F91089502E000936F00FC8EFD8E7D
:1012F00008950F93F0928500F092840078940FB7D0
:101300001F930F93BF93AF9391FD02C01C9B87DF88
:101310001D9B0E940117AC8DBD8D0A2F0B2B31F048
:101320001197AC8FBD8F11F4E0929D020D850023C3
:1013300029F00A9511F490680E850D8709890A95A0
:1013400011F490640FE0098BAF91BF910F911F9141
:101350000FBF0F9118950F93F092B00007E0009324
:10136000B10001E60093B30002D00F91089502E0AE
:1013700007BB02E00093700008950F930FB70F931F
:10138000F092B20000918704002319F008810395C0
:1013900008830F910FBF0F9118950E94F416222712
:1013A000E0E0F1E014E0002721930A95E9F71A95AF
:1013B000D1F7CEE9D2E0FF24EE24E39499278824E4
:1013C00099240FEF0F8F0AA708E208A30FE409A3DF
:1013D00028E02F87EAE7F4E0E0930001F0930101B1
:1013E00000E20BABA0E4B1E0E4E5F0E016E3110F9E
:1013F00005910D931A95E1F7E0929D020EE30D879A
:101400000E870FE0098B05E00B8BEAECFAE0EDA705
:10141000FEA701E800936400F7DE48DF9CDF68D197
:101420000E9446180E946E140E9478140E94BB19F4
:101430000E9405155ED467D40E94D2140E9417152D
:101440000E940D170090F702002011F00E941E1755
:101450000E9439180090E402002031F40090EE025E
:10146000002011F40E9454190E94D3180E94F01811
:1014700054D474D4F6D20090E402002079F4198197
:101480001F93A8D00E94C8181F9109810117C1F3AA
:101490000A9509837CD29FDEE0928704789401D577
:1014A000ACD20E94601A0E94571B0E94601A92D010
:1014B00095FF25C09F7DE9EFFAE0EDA7FEA70E940A
:1014C000A81200E50E949212A8E4B1E00E948712DF
:1014D000F8DE8CD0F6D595D709A10F3441F0FBDEAC
:1014E0000023B9F70E949B120FE40E949212EAECCB
:1014F000FAE0EDA7FEA70FE409A3E0929D0293FF97
:1015000037C0977FF88A0E9444160091F102073194
:1015100011F402EC11C0F09287040E949314009120
:10152000F102083111F009EA07C00091F2020D3012
:1015300011F40CEB01C00DEADDD7C3DE4BD0C1D5F1
:10154000DBD608A1083239F0C6DE0023B9F7CBD7C5
:10155000ACD737D753D70091F102073121F0E09291
:1015600087040E949514E0929D020E2D0E944C1B50
:101570000090F702002011F0ADD599CF90FD0E94A8
:10158000621A95CFFF93EF93EDA5FEA50995EF9114
:10159000FF9108950F921F920F931F932F933F93E4
:1015A0004F936F938F93BF93AF93FF93EF935F939B
:1015B0007F9310D07F915F91EF91FF91AF91BF9199
:1015C0008F916F914F913F912F911F910F911F908C
:1015D0000F9008950090FC02002029F000917F04F4
:1015E000077009F452D3E2D024D0089518D121D045
:1015F00008950F921F920F931F932F933F934F9332
:101600006F938F93BF93AF93FF93EF935F937F930A
:10161000EDDF7F915F91EF91FF91AF91BF918F913E
:101620006F914F913F912F911F910F911F900F90AC
:10163000089592FF21C01D850E949514011B19F089
:101640000E3108F406C00BA800FC02C0A0D101C0F6
:10165000D6D11091FD0210FF07C011FF0E94AB14FC
:1016600012FD0E94B11407C0A8A5B9A50A2E0B2A25
:1016700011F00E94AB149B7F97FF0AC0F8820E9472
:1016800098140BA800FC02C082D101C0B8D19F778A
:1016900096FF03C00E94C2199F7B94FF28C00B894C
:1016A0000A9519F40E94B11405E00B8B0090EA0230
:1016B000002019F00E2D0E944C1B9F7E0FAD01FFE4
:1016C00016C01091EA020091E90210230091EF0286
:1016D000102351F00B81043039F4A0E3B1E0E0ECC9
:1016E000F1E000EF0E9483190FAD0D7F0FAF089559
:1016F000389A399A3A9A3B9A209A219A229A239AAE
:10170000539A549A559A5D9A579A5C9A5F9808959D
:10171000582F580D5B0D5B9855B9529558B95C9888
:101720005C9A562F590D5C0D5B9A55B9529558B974
:101730005C985C9A5D985D9A0895562F580D5B0DE4
:101740005B9855B9529558B95C985C9A582F590DC9
:101750005C0D5B9A55B9529558B95C985C9A5D9846
:101760005D9A0895382E462E880F880D8B0D660FD2
:10177000690D6C0D0AD0839508D08A95639505D0C4
:10178000839503D0642D832D08955B9885B9829548
:1017900088B982955C985C9A5B9A65B9629568B9DC
:1017A00062955C985C9A5D985D9A08951F85A0E0AB
:1017B000B1E0ED91FD91BD90CD900E2E0F2A09F074
:1017C0003AD01A95B1F70888002041F4A0E2B1E0C0
:1017D00015E00FD0A4E3B1E013E016D0A0917F0490
:1017E000B09180041196A0937F04B09380045F9819
:1017F0000895ED91FD91BD90CD900E2E0F2A09F028
:1018000082D01A95B1F70895ED91FD91BD90CD90DC
:101810000E2E0F2A09F070D01A95B1F70895A0E4A2
:10182000B1E01AE1E6DF1E2DEFDF10917F04139582
:1018300010937F040895BF93AF9385918823E9F3B4
:101840008B3071F065914591442309F4F6CF4F3FF9
:1018500089F025912F934F9310D08F916F91F3CFF3
:10186000C59005912B2D56D058D0B22E85918F3F23
:1018700009F0E4CFAF91BF910895DF01E8E8FBE004
:10188000522F561B08F45195042F081B08F401959C
:10189000051740F4EDE9FBE08627682786274227F5
:1018A00024274227481730F48427482784276227B3
:1018B00026276227442E481A522E561A08F45194AD
:1018C000222433246624621710F4639401C06A94BE
:1018D000481778F05F9A0995250C3F1C722D720D00
:1018E00074153F041CF0660D24183F0883954817B3
:1018F00090F75F98FD0108950DD00191002311F03C
:101900000CD0FBCF089506D00591002311F005D02F
:10191000FBCF08954EED5EE008950F0107FD24C052
:10192000015208F15F9AE02FFF27EE0FFF1FEE0F25
:10193000FF1FEE0FFF1FE40FF51F68E0659088277B
:1019400067FC10DF839566FC0DDF839565FC0ADF7D
:10195000839564FC07DF839563FC04DF839562FC59
:1019600001DF6A9559F70F5D5F98F00102D0B00E64
:1019700008950A3311F408E009C0003811F404E0B6
:1019800005C00D3211F40AE001C00CE00895A9D79A
:101990001981139519831C3359F00A8D002311F016
:1019A000FA8E2BC069D008A1007441F5D4D026C0AE
:1019B0009061F9821A8113951A831C339CF01FAD34
:1019C00012601FAFFA821B8113951B83183154F0EC
:1019D000FB8208A1007411F40E94B2151BA911FD2D
:1019E00060D20BC01BA911FD08C00E940E1908A1EE
:1019F000007419F40E94F01854D233D0089571D7AE
:101A00000E850D8719811A9519831F3F41F00A8CA5
:101A1000002011F0FA8E17C02FD09DD015C01BE307
:101A2000198390611A811A951A831F3F61F41BE391
:101A30001A831FAD12601FAF1B811A951B831F3FB6
:101A400011F417E11B830DD008950E946616002340
:101A500029F40E94D3180E94F01803D008950E9420
:101A6000D31831D105D077D008950E94F018F9CF5E
:101A700003D022D041D008950091F2020D3059F0E8
:101A8000EAE7F9E0098115E0019FE00DF11D8F0102
:101A9000E8E0F1E05CC009810E94E716EAE2F3E0C9
:101AA0000AD1E8E0F1E000831183022FE2E7F3E0DE
:101AB00002D1ECE0F1E04BC00091F2020D3059F0A0
:101AC000E6EAFAE00A8119E0019FE00DF11D8F01BD
:101AD000E0E1F1E03CC00A810E94E716EAE2F3E0AF
:101AE000EAD0E0E1F1E000831183022FE2E7F3E0C6
:101AF000E2D0E4E1F1E02BC00091F2020D30B9F048
:101B0000E2ECFCE00A811CE00E94BD160F930B8101
:101B10000E94BD16022F25E0029F1F91100D29E0A3
:101B2000129FE00DF11D8F01E8E1F1E010C00B8183
:101B30000E94E716ECE0F3E0BED0E8E1F1E00083BC
:101B40001183022FE2E7F3E0B6D0ECE1F1E000838D
:101B50001183D5D40895ACEAB1E03091F102383167
:101B6000A1F1373111F4BDD730C00B81363149F0C6
:101B7000343139F40F01E2E2F4E0E00FFF1D04918B
:101B8000F0014ED00AE30D930A814AD00AE30D9387
:101B9000098146D03091F102343151F400E80D93BF
:101BA00011E40B810C300CF010E51D931DE41D9326
:101BB0000090FC02002049F0353111F0363129F453
:101BC0001AE31D9310E21D931D93FD9232D00CA9D0
:101BD000002311F1ECEAF1E0A8EBB1E01CE0019187
:101BE0000D931A95E1F71C970CA910E2013091F0C2
:101BF000023079F0033061F0053031F0043009F043
:101C00000BC013961D9306C017961D931D9302C01B
:101C1000139613961D931D9308950CAB9CDF0895A6
:101C2000802F3091F102363111F451D701C04ED7D7
:101C30000895A8E3B1E0ECEAF1E0ED93FD930AD159
:101C40000D930093E70209E40D930895A8E3B1E032
:101C5000FD92FD92FD92FD9208950090FC020020FD
:101C600069F0ACE3B1E0E4ECF1E0ED93FD930091B9
:101C7000E702005A0D9309E40D930895ACE3B1E037
:101C8000FD92FD92FD92FD9208950091F1020531C1
:101C900011F0063179F4A4ECB1E008810695043620
:101CA00014F0045600000BA800FE02C001950C5968
:101CB000B7DFFD920895000FE00FFF1D059114910D
:101CC000000F111F0895EDA9FEA90091F10208313E
:101CD00011F0073129F40B810C3010F0EFA9F8ADA9
:101CE0000091F2020D3021F0E0930401F093050120
:101CF00008950091F102043110F0093118F004E167
:101D00000093F10208950091F2020A3010F00F30B2
:101D100018F00AE00093F20208950091F1020F9387
:101D2000083189F0043131F0053139F0063129F0FC
:101D3000073101F0A3DF0FDF08C00DDF8EDF05C024
:101D40009DDF09DF02C082DF99DF0F9108950093C4
:101D5000F102E3DF38D6B7DFFEDE08950091F2022C
:101D60000A3049F00B3051F00C3079F00D3029F188
:101D7000E6E1F9E00CC0E6EAF5E009C0E6EAF5E0E4
:101D8000EDABFEABE4E9F6E004C0E8EFF7E0EDAB65
:101D9000FEABEFABF8AFE6E2F1E009E7019304EB4D
:101DA000019332960BE6019304EB0193329607E818
:101DB000019304EB01935BD011C0E6E2F1E009E787
:101DC000019301E0019332960BE6019301E0019348
:101DD000329607E8019301E001930BD042DE0895AB
:101DE0000093F202BBDF0091F202E7D56CDF40DE28
:101DF0000895EAE0F1E018EB108334961FEC1083AD
:101E000034961EE61083349615E81083349610E25B
:101E10001083349617E31083E6EEF2E0E0930001BE
:101E2000F0930101F0920401F092050119E101D053
:101E30000895A4E3B1E00090F902002041F4E7EC3A
:101E4000F1E0ED93FD9306D00D931D9302C0FD923A
:101E5000FD92089522270191002329F08ADD200FA9
:101E6000D0F7002703C00FEF021B0695089506E088
:101E7000E8E0F1E0F192F192F19231960A95D1F712
:101E8000F0923401F092350111E9D3DFEAE7F4E092
:101E9000E0930001F093010116DF0895F0928604AB
:101EA00002C0E0928604EFE9F2E029D0C5D058F0F4
:101EB00066D00023B1F40091860400FD0E949D15B8
:101EC0007AD0EFDF0EC0E6D060F059D0002349F0A1
:101ED00061D0002331F40091860400FD0E94A71513
:101EE0007ED008950091F402023039F00581085047
:101EF00020F0083010F48894089508940895009113
:101F0000F402003059F0013009F1F0928104F092AE
:101F10008304F0928404F09282040895E3DFA8F32E
:101F200012E0109381041BE0109382040F01E6ED90
:101F3000F2E0E00FFF1D0491F001102F12951F70C9
:101F4000109383040F70009384040895CBDFE8F2AC
:101F5000E09281041AE0109382040F01EFE6F1E0B1
:101F6000E00FFF1D0491F001102F12951F70175EF6
:101F7000109383040F70075E009384040895EFE9C3
:101F8000F2E000C0AFDF10F400270895102F009199
:101F9000F5020AC0EFE9F2E000C0A4DF10F4002768
:101FA0000895102F0091F602112319F01A95069545
:101FB000FBCF01700895EFE9F2E000C093DF10F469
:101FC00000270895102F1FD01091F502102B1093A9
:101FD000F502012F0E94E7140E941A1A0895EFE9F2
:101FE000F2E000C07FDF10F400270895102F0BD01F
:101FF0001091F602102B1093F602012F0E94E914A3
:102000000E941A1A08950E2D112319F01A95000F27
:10201000FBCF0895E5EAF2E072DF0ED078F0009091
:102020008504002039F0B9DF002341F4E5EAF2E04D
:10203000D9DF04C08894089555DF10F408940895FA
:1020400004810330D8F3B9F010918204011700F134
:10205000A9F70381109184040117D0F079F7028168
:10206000023010F008940895F0928504013080F059
:10207000E09285040DC00381109183040117F0F2F2
:1020800039F4028110918104011710F40894089525
:102090008894089527DF10F408940895048110911E
:1020A0008204101760F0C1F70381109184041017A7
:1020B00030F091F70281023010F40894089588946A
:1020C000089500917E04002321F00E94CA17F09227
:1020D0007E04089500917E04002349F000919D0242
:1020E000002379F30E946616002359F701D0089562
:1020F000F0927E0433E6A8E3B2E00E94AD17A8E3B5
:10210000B2E0E8EBF2E20E94521100FF7CC002E074
:102110000E9443110C91013409F075C0F0929D02A8
:10212000D7D80091E902002311F404E074D001E053
:102130000E944311C5D08987C3D08887C1D08F83BF
:1021400009E00E944311BCD08A87BAD08B87B8D0EF
:102150008C8709850090F802000D09871CF0083172
:1021600030F409C0085E09870E94231104C0085199
:1021700009870E941E114EDF10F00E942811098568
:102180000B80001549F408850A80001529F40F8199
:102190000980001509F409C009840B8208840A82A9
:1021A0000F8009820E940E19EA8E0C850E800015A0
:1021B00049F40B850D80001529F40A850C80001563
:1021C00009F409C00C840E820B840D820A840C82EF
:1021D0000E944A19EA8E0A8C0020A9F05FDEA4E270
:1021E000B1E0E2E0F2E00E9487190A2E0B2A49F0E2
:1021F00005E0A00FBF1D04E10D931296FD92FD9224
:1022000002C004E101D00895A4E2B1E0E2E0F2E00E
:102210000E9483190895A4E2B1E0E2E0F2E00E9496
:1022200087190A2E0B2A49F4A4E2B1E002E0002E3D
:1022300002E0102E04E00E9462190895E5EAF2E03F
:102240000E94BA150895E5EAF2E00E94C2150895C9
:102250001985139518311CF0F986F0DF11271987BD
:102260000895E5EAF2E00E94DA151395011708F0E7
:1022700000270895FF93EF93E5EAF2E00E94DA1554
:10228000EF91FF910895A8E3B2E01127002E039487
:102290000A9439F00D9113950A3019F00C32C1F3FC
:1022A000F9CF08950D910590001521F40C32D1F766
:1022B0000E2D01C000270895244750524D432C0095
:1022C0000D911D910295007F1F70012B802F0E94A0
:1022D000D51608950E94DF170090F702002019F428
:1022E0000E941E1702C00E9425170E240092F702BA
:1022F000002D0E94ED140895E8E5F2E008A12FD02A
:1023000008A30590001611F03596FBCF95FF07C086
:102310009F7D319605911491F80109951DC093FF99
:102320001DC005911CD0E6D00E946109329605912E
:102330001491002E012A81F017FF02C06EDC0CC040
:1023400016FF08C01F7B0F931F93D8011496C7D0A8
:102350001F910F91D801B8D00E9461090895102FE4
:10236000107811F090620F770895A0E2B1E004E3D5
:102370000D9301E00D9307E30D930DE20D93149778
:10238000089577D002C0F1DF90D098600895098158
:1023900003950C3308F0002709830DC00A810395CB
:1023A0000C3308F000270A8306C00B81039508311F
:1023B00008F000270B8355DB089530D70E944E0F9D
:1023C00001C0F1D608E296D0F0922001F0922101EE
:1023D00048DB089515D4EFCF0C8108D4002311F405
:1023E0001A951C83986008950FD4E5CF11D4E3CFDC
:1023F0005CD050D70E94510F98600895F1D631DB20
:102400000895E4E0F2E009A10D3541F41091E002F5
:10241000123009F403C00FE485D008950055002E52
:10242000000C000C000F000DE00FFF1D95FF06C013
:102430009F7D05901590F001099517C093FF17C077
:10244000329605901590FF93EF93F001099509A13D
:1024500003950E350CF00FE465D0EF91FF91A59137
:10246000B5910A2E0B2A09F052D00E9461090895F5
:102470000895A8E3B1E0ECEAF1E008EB002E01E0FA
:10248000102E0FEF0E946219AFA7B8AB0895A8EA0B
:10249000B1E0E7ECF1E00CED002E01E0102E0FEFC3
:1024A0000E946219AFA7B8AB0895AFA5B8A90E9462
:1024B000A519FFA6F8AAFCAA0895ED91FD9112971F
:1024C0000FEF0E9483190895F8DFAAA3BBA3089514
:1024D000AAA1BBA10E94A519FAA2FBA20895EDDF53
:1024E000ACA3BDA30895ACA1BDA10E94A519FCA2F7
:1024F000FDA20895977F08A3EBDFF5DF0895AAA159
:10250000BBA10E94F419ACA1BDA16ED70895D5DF7F
:10251000AEA3BFA30895AEA1BFA10E94A519FEA2BC
:10252000FFA20895977F09A3F6DF0895AEA1BFA18A
:102530000E94F41908951091E002123011F4B5DFF1
:1025400001D0089574D20ADC08958DD207DC089575
:10255000088909AF6DD01091F1021DAF4FD00091E5
:10256000E9020AAF76D00091EF020BAF84D0009160
:10257000F2020CAF2DD00BA80EAE92D00090F90253
:102580000092E002A4D00090FC020092DE027FD113
:102590000090FA020AAAF9AABDD0C8D00CE30090B4
:1025A000F702002019F00091F802075B00939C02EB
:1025B0001AD10091F4020093DF0253D1F092E102AC
:1025C0007CD108950CAD03950F300CF00AE00CAFF0
:1025D0000CAD0A50E4ECF1E06EDBE4E5F1E021C083
:1025E0000CAD1091F202011711F0FADB17D008952B
:1025F0000DAD039509310CF004E10DAF0DAD0451A3
:10260000EEECF1E058DBECE4F1E00BC01091F102EC
:102610000DAD011711F09BDB01D008950DE509A365
:1026200008950083118382DF089509AD0E2509AF57
:1026300009ADE8EDF1E03FDBECE7F1E0F2CF09AD09
:102640001889011711F033D3E9DF08950AAD0E257B
:102650000AAF0AADE4EEF1E02EDBE4E8F1E0E1CF11
:102660000AAD1091E902011711F057D3D7DF089591
:102670000BAD0E250BAF0BADE4EEF1E01CDBECE88F
:10268000F1E0CFCF0BAD1091EF02011711F04ED357
:10269000C5DF08950EAD039504320CF000E20EAFD5
:1026A0000EAD0052ECEDF1E006DBE4E9F1E0B9CF6C
:1026B0000EAD1BA9011711F01BD3B0DF08950091D7
:1026C000E002039503300CF000E00093E00200917B
:1026D000E0020050E4EEF1E0EEDAE4EAF1E0A1CF4E
:1026E0000091E002023019F4F9AAD1DE06C010917F
:1026F000F902011711F009D391DF089509A9E7EC58
:10270000F1E0E00FFF1D0081039507FD00E200836B
:102710000DD00895E7ECF1E00F010AA9E00FFF1DCD
:10272000F082F00197DB0093AA010895E7ECF1E055
:10273000ACEDB1E014E101910D931A95E1F709A90F
:10274000ECEDF1E0E00FFF1D0FE50083089509A90E
:10275000039509AB03951AA901170CF00AAB0A956A
:1027600004316CF0E7ECF1E00A9531F0E00FFF1D69
:102770001081103209F4F6CF039509AB1EC0E7ECC7
:10278000F1E00A9559F00A95E00FFF1D1191103202
:1027900029F41191103211F409AB0FC009A9E7EC2B
:1027A000F1E0E00FFF1D0081002311F400E200833F
:1027B000B1DFBCDF0CE509A3089509A90093FA0273
:1027C000E7ECF1E0E00FFF1DF082F092E602BDDEE3
:1027D0006CDE24DF089500919C02039506350CF011
:1027E0000CE300939C0220919C022C5306E411E020
:1027F000220F220F020F1F1DECE5F1E012CF009116
:102800009C020C3391F009541091F702112321F02E
:102810001091F8020117E1F00093F802E092F7023C
:102820000E94DF170E941E170CC0F092F802109150
:10283000F702112369F0F092F7020E94DF170E945D
:1028400025170091F702C9D00091F802C8D0E6DE42
:1028500008950091DF02039503300CF000E000932F
:10286000DF020091DF02EAEEF1E025DAE4E6F1E0D2
:10287000D8CE0091DF021091F402011711F06ED250
:10288000CDDE08950091DE020E250093DE02009158
:10289000DE02E8EDF1E00FDAE4E7F1E0C2CE00910C
:1028A000DE021091FC02011711F051D2B7DE08953B
:1028B0000091E1020E250093E1020091E102E8EDB2
:1028C000F1E0F9D9ECE9F1E0ACCE0091E1020023AE
:1028D00021F0EBD00E940117A1DE0895569A5E9870
:1028E00008950091E90200FF4E9A08955E980895B8
:1028F00024982C9A08950AA50F3F71F4EAA6A09196
:10290000E202B091E3020A2F0B2B31F400EF05D065
:10291000A093E202B093E3020895A8E2B1E0EEEFE3
:10292000F1E0F1D40895FD8608950E850D87089590
:102930000BA901FD0895A8A5B9A50A2F0B2B21F419
:102940000FEF03D0A8A7B9A70895ACE2B1E0E0E08B
:10295000F2E0D9D40895A8A5B9A5F7D4F8A6F9A6A8
:1029600008950A890F3F61F00F01EAE3F4E003954F
:1029700007700A8B000FE00FFF1D85909490F00107
:1029800008950090EF02002021F40090E5020A8AE9
:10299000E8DF08950A890093E5020FEF0A8B882487
:1029A000992408950888002039F40091EF0200234B
:1029B00011F0F0DF01C0E5DF0895A9E01DC0A0E03F
:1029C0001BC0A6E019C0A8E017C0ABE015C0ACE082
:1029D00013C0ADE011C0A1E00FC0AEE00DC0AFE08C
:1029E0000BC0A5E001E008C0A0E106C0A2E104C060
:1029F000A3E102C0AAE000C00090FD02002021F483
:102A0000BB2700BD16E0AFD10895ADEFB2E0E9EE0F
:102A1000F2E0AE1BBF0B2A2FA0E0B0E011E0A3D183
:102A20000F3F09F4002701932A95C9F70895E7ECB1
:102A3000F1E00091FA02002349F0202FAEE1B0E06E
:102A400011E091D101932A95E1F70CC0DF01E0E09C
:102A5000FBE32BE02093FA0205910D932A95E1F711
:102A6000E092E60208950090FD020020E9F4009053
:102A7000E6020020C9F40091FA02002331F400E2DA
:102A80000093C7010E2D0093FA02202FA1E1B0E0C0
:102A900000BD16E068D1AEE1B0E0E7ECF1E00191F5
:102AA00000BD61D12A95D9F70895ADEFB2E0E9EE06
:102AB000F2E0AE1BBF0B2A2FA0E0B0E016E00FEF54
:102AC00000BD51D1F1922A95D1F708957AD18F9313
:102AD00082958F7081D18D938F918F707DD18D93E1
:102AE0000895EFE9F2E08381F1DF8DE28D93848137
:102AF0000F01EAE4F4E08A95880F880FE80FFF1DC4
:102B000085918D9385918D9385918D938DE28D9394
:102B1000F00182E38D9380E38D938581D7DF089563
:102B2000EFE9F2E08281D2DF8AE38D938181CEDF0B
:102B30008AE38D938081CADF08951B8113951B83DF
:102B400018311CF0FB8216D0A5D368D308951B81E1
:102B50001A951B831F3F21F417E11B8313D09AD3CF
:102B60005DD30895EFE9F2E005D00895EFE9F2E0D2
:102B700009D008955AD00E1521F461D00E1509F42C
:102B800067D0089503810A95038359F404810A9557
:102B9000048329F40CE0048305810A9505830AD097
:102BA00013830895FF93EF93EFE9F2E003D0EF91E1
:102BB000FF910895BF93AF930F930481AAE4B4E00B
:102BC0000A95000F000FA00FBF1D1396FF93EF9300
:102BD000FD011491EF91FF911C3121F405810370E7
:102BE00009F41DE10F91AF91BF910895EFE9F2E073
:102BF00001D00895DFDF1395011708F0002708952D
:102C0000EFE9F2E012D00895EFE9F2E018D008956C
:102C1000EFE9F2E01DD00895EFE9F2E008C0EFE936
:102C2000F2E00FC0EFE9F2E015C003810395002345
:102C300019F0E0DF002309F40E2D038308950481C9
:102C40000395002311F00D3008F00E2D0483089534
:102C500005810395043608F0002705830895082FA1
:102C60000C3310F48983089500270895082F0C333E
:102C700010F48A83089500270895082F083110F46E
:102C80008B83089500270895F4D17BDE18E01F8719
:102C900065D8089522D0E9D17DDEEF86E2EFF2E03B
:102CA000E0930001F0930101089508890E25088B37
:102CB000002311F0EFDF01C0E7DF4EC00091F30207
:102CC0000E250093F30296DE9CD046C00BA900327D
:102CD00011F4002701C00E2D08950BA901FF03C0B8
:102CE0000EE30E870D8700E20BAB0E94250D0895C1
:102CF0001BA9102711FF05C01EE301FD12E01E876E
:102D00001D870BAB0E94250D08950093F9026CDE20
:102D100025D808950091E9020E250093E90200FDEF
:102D2000E5DD4DDE19C00091EF020E250093EF02A4
:102D30000F9347DE0F9136DE0FC00091EA020E2599
:102D40000093EA0248DE08C00091FC020E250093C1
:102D5000FC024EDE0E948D0E889408950093F402CA
:102D600034DE9FD80895A1BDB2BD119611FDFA9A27
:102D70001FBBF999FECF00B50895222738E0000F58
:102D8000221F211710F00395211B3A95C1F70895D2
:102D9000202F1AE1019F1A941AE0012D019F20199A
:102DA0002A3010F02A50039508950F938F9382953F
:102DB0008F700AE0809F002D8F918F70800F0F9190
:102DC0000895082F04D00295022B802F0895E0DF8C
:102DD0000A300CF00E2D08950F01E2E1F4E0E80F47
:102DE000FF1D8491F0010895A89504B7077F04BFE3
:102DF000009160000861009360000027009360006C
:102E00000895F894A895009160000861009360000F
:102E10000AE0009360007894089510E41093C400D1
:102E2000F092C500F092C00018E410691093C10040
:102E300016E01093C200EC8AC2D0089513E01093FC
:102E4000C40011E01093C500089510E41093C4006D
:102E5000F092C50008950F930FB70F931F93FF9340
:102E6000EF930F890F3F79F00395EEEFF2E0E00F5B
:102E7000FF1D1081112319F40FEFEC8A02C010938B
:102E8000C6000F8B11C0ED89FE890E2F0F2B31F07C
:102E900031961491112321F4FD8AFE8AEC8A04C034
:102EA0001093C600ED8BFE8BEF91FF911F910F9158
:102EB0000FBF0F9118950F930FB70F931F932F9379
:102EC0003F93FF93EF932091C600088D302F039519
:102ED0000F77198D011731F40091F70200FDE09290
:102EE0007E040EC0088FEEEFF3E0E30FFF1D20839A
:102EF00091602A3029F42091F70220FDE0927E04AF
:102F0000EF91FF913F912F911F910F910FBF0F9163
:102F100018950F930C890023E9F3FC8A8093C6006F
:102F20000F91089590FFFECF0F931F93FF93EF93A0
:102F3000188D098D8827011751F0EEEFF3E0E00FAF
:102F4000FF1D808103950F77098F011709F49E7F7C
:102F5000EF91FF911F910F9108951127F894288DFB
:102F6000098DEEEFF3E0E00FFF1D808103950F77F1
:102F70001395131708F011978D938A3029F00217D3
:102F800081F79E7F8AE08E93021709F49E7F098F56
:102F900078940895F894288D098DEEEFF3E0E00F12
:102FA000FF1D808103950F778A3019F00217A9F76A
:102FB0009E7F021709F49E7F098F789408950FEF82
:102FC0000F8BFD8AFE8A08950F939E7FF88EF98EEF
:102FD000F0927E040F9108950F93FF93EF930C8965
:102FE0000023E9F3FC8AED8BFE8B04910093C6006D
:102FF000EF91FF910F9108950F93FF93EF930C8939
:103000000023E9F3FC8AFF8AEEEFF2E0008100235F
:1030100021F40FEF0F8BEC8A02C00093C600EF91F2
:10302000FF910F910895889490FD08940895089455
:103030000C88002009F4889408951F930F9319D0E9
:1030400003D00F911F9108951FE000E444D01EE0CB
:1030500001E841D011E001E13ED008951FE000E415
:103060003AD011E001E137D008951DE000E833D0F7
:1030700008951DE000272FD00895000000000000F3
:10308000000000000000000000000895449A459AE6
:1030900008953F9333273A9519F4E092E40217C05C
:1030A000B1F06AD0EADF02EA3FD0E7DF33D098F32D
:1030B000012F3AD0E2DF2ED070F355D05DD003EA75
:1030C00033D0DBDF27D038F33CD0449A459A4BD03D
:1030D000802F3F9108953F9333273A9519F4E0925A
:1030E000E40215C049D0C9DF0F9302EA1DD0C5DF45
:1030F00011D00F9190F30F93012F16D00BD00F9199
:1031000060F30F9311D006D00F9138F300002BD04D
:103110003F9108953C98449A0894459AAEDF349BB9
:10312000889445983C9A08953F9338E0449A000F5C
:1031300008F04498459AA1DF45983A95B9F73F9130
:1031400008953F933C98449A002738E0459A0894A4
:1031500094DF349B8894001F45988FDF3A95B1F730
:103160003C9A3F9108954498459A00000000449A83
:1031700000003C983D9808953C9A3D9A449A459A9F
:1031800000000000449800000000459800000895E9
:103190008F9312E07EDF8F7708DE8C330CF0882768
:1031A00089838F9108958F9312E073DF87FDA3DBEE
:1031B0008F77FBDD8C330CF08827898313E069DF80
:1031C0008F77F3DD8C330CF088278A8314E061DF7E
:1031D0008F73EBDD88310CF088278B838F910895F6
:1031E0000F938F9315E055DF8F73DFDD80320CF086
:1031F0008E2D8C8317E04DDF8F71D7DD882311F082
:103200008D300CF08E2D8D8318E043DFCEDD8436BB
:103210000CF088278E838F910F9108958091FD0285
:10322000882331F4898105D08A810DD08B8113D018
:1032300008958F93082F0C3320F48983C2DD12E0A8
:103240004ADF8F910895082F0C3320F48A83B9DD6B
:1032500013E041DF0895082F083120F48B83B1DD9E
:1032600014E039DF0895C2DC002329F00C83802F9D
:10327000A8DD15E030DF0895082F0D3020F48D8390
:10328000A0DD17E028DF0895082F8E839ADD18E06F
:1032900022DF08950C81E7DF002309F4A1DF8D818F
:1032A000EBDF8E81F1DF08958827C3DF8827CBDF2E
:1032B0008827D1DF01E0D7DF81E0DEDF8827E4DF88
:1032C00090DB0895BF93AF93A2EFB1E016E02D918C
:1032D0003D91232B31F018961A95C9F7EF91FF9184
:1032E00011C0ED93FD93ED920D93EF91FF9101913C
:1032F0000D9301910D930D921D921A973297ED93B4
:10330000FC931197089500241124DCDF08954F9356
:103310005F93AD01A2EFB1E016E02D913D91022E39
:10332000032A61F02417350739F42D913D912E17AA
:103330003F0719F4149706C0129616961A9569F766
:10334000AA27BB275F914F9108950A2E0B2A69F097
:10335000FF93EF93ED91FD9114960D911D910193C3
:103360001193189703D0EF91FF9108950AE0FD9211
:103370000A95E9F7089517E0A2EFB1E0F7DF1A9593
:10338000E9F70895A2EFB1E026E0BF93AF930D9166
:103390001D91012B21F012972F9307D02F91AF9100
:1033A000BF911A962A9589F708950D911D9112964D
:1033B0002D913C913F3F19F03A953C9371F0322F9B
:1033C0003E253E93222311F0149601C012972D91B1
:1033D0003D91D8012D933D9306C01597FF93EF9330
:1033E000B4DFEF91FF9108954A2F4B2B59F04D9187
:1033F0004E1741F44D914F1729F40D931D931296DA
:103400000D931D9308953BD1FE92FE9256D0AAEAE9
:10341000B0E002C0A2E3B0E011E0A5DC002349F077
:103420000F3F39F0BF93AF93802F3ED0AF91BF9144
:10343000F3CF66C0EAECFAE3AEEFB2E032D104D0EB
:103440002CD1FD923AD0089506E48091F50208D07F
:1034500002E48091F60204D0089580E28D930895ED
:103460000D9335DBFADF0895813624F08B3710F4A5
:1034700000E2801B08950C94C20AD9DD10F0FBDF36
:10348000FCCF08950F9309818EE1080F0C330CF0E7
:103490000C53C9DD28F0EFDF8981081721F0F9CF3F
:1034A00041DD0F912DC02EC08F93E7DF8F9131DD6D
:1034B0000895FBE3E2DF90DD0895DFDF9DDD0895F1
:1034C000E2EEF7CF2FDDD0DF8835B9F4E0EAFAE39A
:1034D000F1DFD8DFE9DFC8DFF3DF8154BCF38A31E5
:1034E000ACF7880FECE6FAE3E80FFF1D05901590A6
:1034F000F001099510F4E0E9DCDFDBD0EA8E0895F5
:103500008894089508940895E2EAD3DF0895ECE2E0
:103510009CD0B8F0B2DB0817A1F4D2DFEAE395D073
:1035200080F0A4DB081769F4CBDFEAE48ED048F022
:1035300096DB081731F472DE0E944E0F0E94310DA7
:1035400038C00E942F0DDECF0091EA02002321F047
:103550002ADE46DE0E94310D92D0D2CFEAE575D048
:10356000D0F0082F5FDB0817B1F4AADFECE66DD0CE
:1035700090F0082F54DB081771F4A2DFEEE765D056
:1035800050F0082F49DB081731F484DE0E94510FF8
:103590000E94310D0EC094DF0E94350DB3CFB4DF11
:1035A000E2EB53D040F0853030F48C5E082F0E945F
:1035B000A70E86DFA5CFA6CFA7DFE2EB46D038F077
:1035C000853028F4865F082F0E94F00EF2CF9ACF44
:1035D0009BDFEAEB3AD028F0833018F4082FBEDBEB
:1035E000E8CF90CF8DCF90DFE2EC2FD030F0843059
:1035F00020F4805E082F7CDBDCCF84CFE0ED59DF48
:103600007FCF53DA0E9401177BCFEAEC52DF1127FC
:10361000A7ECB1E037DF98F047DF8D9313951431B5
:10362000CCF38E91803211F41A95D9F71196FC9251
:103630001093FA02F092E6020E94A51261CF0E9456
:10364000A21260CF0E9401175BCF33DF1BDF2CDF9C
:10365000883509F457CF0CD0C8F3082F13DF24DFC7
:103660008835C1F305D0D0F31AE0019F800D48CF13
:10367000803320F08A3310F4805342CF43CF0F8938
:103680000F3F49F4AEEFB2E0E0E00AD0E2E108D04B
:10369000ECE006D002D008950CC0E2EE01D008950F
:1036A000FBE305900D920020E1F711970895E7DF05
:1036B00002C0AEEFB2E00F890F3F09F038C011DA57
:1036C000CCDE2EDACADE0091E902002311F48CE48C
:1036D0008D930091EF02002311F482E48D93009109
:1036E000EA02002311F086E58D930091F402023086
:1036F00029F085E5002309F085E48D930091FC0213
:10370000002311F08BE48D930BA9003211F086E4B5
:103710008D930889002311F083E48D939EDE94DE5F
:103720000DE48091F3029CDEB8DFFD92C6DE0895C1
:103730000027A7ECB1E005900D9203950020D9F782
:103740000A950093FA02F092F9020E94AE0E0895D3
:103750000E94680995FF02C09F7D53DB0E94C20A48
:103760000E9461100E946B090023A1F70895E0E216
:10377000F1E0A8EFB1E0A193B19309E601930DE266
:103780000193ABDA2CD030D0EAECFAE0EDA7FEA73B
:103790005CD0E0E0FBE3CCDF01D008950FD004D093
:1037A000D7DF089508E107C004E105C005E103C0C3
:1037B00006E101C007E10E94A70E1BC00AE007C096
:1037C0000BE005C00EE003C00DE001C00CE00E945C
:1037D000F00E0FC00E2D01C000279FDA0AC000278F
:1037E00001C00E2D64DA05C0002701C00E2DAFDA2E
:1037F00000C00895ABA5BCA5A0E0B1E0EAE7F4E005
:1038000000E581DDABA7BCA70895ABA5BCA59DDDF8
:10381000FBA6FCA6089500E20E940411089500E2B0
:103820007CD8089500E291D80895BEDF91DFC2DF11
:103830008FDFBCDF8DDFDADF8BDFD6DFB9DF88DF3C
:10384000B3DF86DFAFDF84DF08950FE00B830AE28A
:103850000A830E94310D089501E00093FD0287DF85
:103860002FDED8DDE2DFE4E9F9E362DFA7DF70DF16
:10387000A9DF6EDFA5DF6CDFA9DF6ADFE4EAF9E329
:1038800057DFA2DF65DFD1DFECEEF9E351DF90DF38
:103890005FDF94DF89DFE8E5FAE34ADF59DFE4E937
:1038A000F9E346DF55DFA2DF8BDF52DF9DDF82DFEA
:1038B0004FDF8CDF4DDF88DF77DF4ADF83DF78DFA4
:1038C00047DF72DF7BDFECEBF9E332DF83DF40DFE2
:1038D00083DF3EDFEAEFF9E32BDF3ADF82DF38DF19
:1038E0007EDF36DFE2EBF9E323DF02E201DA30DFED
:1038F0002FDFF3D92DDF01E2FBD92ADF29DF03E235
:10390000F7D926DF25DFE9D9E8ECF9E311DF87DF16
:103910001FDF1EDF03E00093FD0284DF19DF18DFE5
:1039200001E00093FD0277DF13DF12DF63DF10DFBA
:103930000FDF6BDFEEE0FAE3FBDE05E00093FD0254
:10394000FA8A06DF05DF01E00093FD02E2EDF9E30C
:10395000EFDE0E94A812E9EFFAE0EDA7FEA7F8DE7D
:10396000F7DEEAECFAE0EDA7FEA7E0E2FAE3E0DE3C
:10397000EFDEE0E3FAE3DCDEEBDEE2E4FAE3D8DEFE
:10398000E7DE0CDFE2EEF9E3D3DEE2DEE1DE0E9409
:1039900001170895596F7572204E616D6520686535
:1039A0007265000042696E61727920436C6F636BCF
:1039B0000000506C6179204D6F6465004C454420D7
:1039C000436F6E74726F6C005761726E696E6773CD
:1039D00000004F6E2053637265656E204D656E75F5
:1039E00000005468616E6B20596F750042692D4864
:1039F000657820436C6F636B000043616C69627291
:103A00006174696F6E2053637265656E0000427564
:103A1000726E496E2050726576656E74696F6E00C5
:103A2000416C736F20537570706F72746564000021
:103A3000475053204E4D45412050617273696E6767
:103A400000004461796C6967687420536176696E1F
:103A5000672054696D650000333020436F6D6269E3
:103A60006E6174696F6E730088940895801A93165E
:103A70005516AE1A341DDC1A6A11031A2C1C221BAF
:103A8000A4168A165E16CF1AFE1AF31A801A011BA4
:103A9000A41A871AE81A9D16051B821A341DF21AF9
:103AA000436F6D6D616E6428422C432C442C462C70
:103AB000472C482C4B2C4C2C4D2C4E2C502C522C43
:103AC000532C542C552C56293A00445354206669E3
:043AD000782000005A
:103B0000447574636874726F6E69780056332E332F
:103B1000610020415652204F7363696C6C6F736370
:103B20006F706520436C6F636B2000003220646906
:103B3000676974206872733A20003220646967698B
:103B400074206D696E733A202000322064696769C1
:103B50007420736563733A202000322064696769BA
:103B60007420796561723A20202020003220646937
:103B7000676974206D6F6E74683A202020003220CF
:103B80006469676974206461793A202020202000EC
:103B90002043616E63656C2F54696D656F75740D9C
:103BA0000A00322064696769742076616C7565204B
:103BB000000028302D34293A000028302D32293ACF
:103BC000000028302D33293A00004E616D65200039
:103BD00028432932303038204A616E2064652052F3
:063BE00069650D0A0000FA
:00000001FF
